:103C43000ECF0EBB0EA70E920E7C0E650E4D0E34DC
:103C53000E190DFE0DE10DC40DA50D850D640D426C
:103C63000D1E0CFA0CD40CAE0C860C5D0C330C0838
:103C73000BDC0BB00B820B540B250AF50AC40A9319
:103C83000A610A2F09FD09CA09960963092F08FC6D
:103C930008C808950861082E07FB07C8079607643C
:103CA3000733070206D206A206730645061705EA7E
:103CB30005BF059305690540051704F004C904A36E
:103CC300047E045A0437041503F403D303B40396A0
:103CD3000378035B033F0324030A02F002D702BF06
:103CE30002A80292027C02670253023F022C021ACC
:103CF300020801F701E601D601C701B801A9019C39
:103D0300018E018101740168015D01510146013C8D
:103D130001320128011F0115010D010400FC00F40B
:103D230000EC00E500DE00D700D000CA00C300BDF0
:103D330000B800B200AD00A700A2009E0099009455
:103D43000090008C008700840080007C0078007560
:103D53000072006E006B0068006500620060005D29
:103D6300005A0058005500530051004E004C004AC1
:103D730000480046004400430041003F003E003C31
:103D8300003A003900370036003500330032003185
:103D9300002F002E002D002C002B002A00290028C4
:103DA3000027002600250024002300010C01010444
:103DB30002011E030A96040132050202060064078B
:103DC300010108000009015A0E01010F0001120050
:103DD3006413010114013C1501FA1664FA17FFFF7D
:103DE3001D00072000072400022701012F013C309A
:103DF300010132010335FFFF3603073CFFFF3DFF9F
:103E0300FF180002191E461A00021B00022D32C8B9
:103E13002E0001FAFAFA18000019FFFF1A00001B1E
:0B3E230000002D32C82E0001FAFAFA50
:10004800900786E0FEA3E0FF7457BE0010D39F40E0
:100058000C903DAD12001EE493F599802F9000148A
:10006800E0D394044014900786E0FEA3E0FF903D9F
:10007800AD12001EE493F5998012900786E0FEA366
:10008800E0FF903DC212001EE493F5999007861296
:10009800000E900786E0FEA3E0FF746C6F4E7003BD
:1000A80075130022900072E0B40208740190007287
:1000B800F0D20C90013AE090002AF090013BE090D9
:1000C800002BF090013CE090002CF0A20AB34016FF
:1000D80090013AE0700C90013BE0700690013CE022
:1000E80060028002C20A90013AE0B4300F90013BEE
:1000F800E0B4470890013CE0643B60028004D20B06
:100108008002C20BE558B40102800302022E90005F
:1001180057E0F566900062E0F568900063E0F569E5
:10012800900074E0F56A90007AE0900029F0900061
:100138007CE0F56590007DE0F567900080E0F5646F
:10014800900081E0F563900090E0900041F090000D
:1001580091E0900042F0900092E0900043F090000F
:1001680093E0900044F0900094E0900045F09000F7
:1001780095E0900046F0900096E0900047F09000DF
:1001880097E0900048F0900099E0900033F09000DC
:100198009AE0900034F090009BE0900035F09000D9
:1001A8009CE0900036F0900079E0B4011790000AC6
:1001B800740FF0A374FFF090000CE4F0A3F0740245
:1001C800900079F0900079E0B4035990000CE0FEBB
:1001D800A3E0FF90000AE0FCA3E0FD120003741006
:1001E800123F8E7408123F80EF900026F0EF7006E1
:1001F80074FF900026F07400900079F090000BE0F6
:10020800900027F090000AE0900028F0900026E087
:10021800900789F0900027E090078AF0900028E086
:1002280090078BF0803F900081E07006755801754B
:100238006300A20AB3402E90013AE090002AF090A1
:10024800013BE090002BF090013CE090002CF090F6
:10025800002AE0700C90002BE0700690002CE06003
:10026800028002C20AE5667003756602E5687003DB
:100278007568027E887F4DE5668E048F05FF123F04
:10028800708C398D3AE56975F0FAA4FFAEF0E5682F
:100298008E048F05FF123F708C3D8D3E90004FE01D
:1002A800F56090004DE0FE900069E0B506189000FA
:1002B8004CE0FE900068E0B5060C90004BE0FE9024
:1002C8000059E06E606F900069E07006900068E089
:1002D80060067400900059F0900069E0B40208903C
:1002E80000497401F08005900049E4F0900068E04E
:1002F800B4020890004A7401F0800590004AE4F0C6
:10030800900068E0600690004AE060028005756031
:10031800038003756004E559B55802D20C90006853
:10032800E090004CF0900069E090004DF09000598A
:10033800E090004BF0740190009EF0740090009FD4
:10034800F074009000A0F074009000A1F074009088
:1003580000A2F074009000A3F074009000A4F07460
:10036800019000A5F074009000A6F074009000A71A
:10037800F074009000A8F074009000A9F074009048
:1003880000AAF074009000ABF074019000ACF07417
:10039800009000ADF074009000AEF074009000AFD3
:1003A800F074009000B0F074009000B1F074009008
:1003B80000B2F07401900362F07400900363F0746B
:1003C80000900364F07400900365F0740090036675
:1003D800F07400900367F07400900368F074009064
:1003E80003A2F074009003A3F074009003A4F074C7
:1003F800009003A5F074009003A6F074009003A782
:10040800F074009003A8F074009003E2F074019077
:1004180003E3F074009003E4F074009003E5F074D3
:10042800009003E6F074009003E7F074009003E88E
:10043800F07401900422F07401900423F074009089
:100448000424F07400900425F07400900426F074DD
:1004580000900427F07400900428F022E5B554F7C2
:10046800F5B5E5B554FDF5B5C2A2C2A1C292C20761
:10047800E5B554FBF5B5755104E55104F552900006
:100488004FE0F560900025E4F0C209E5B554FEF5AB
:10049800B5C28E758D00758B00754C00752600757C
:1004A8002500D28E22750A00750900AE09AF0A74BC
:1004B80057BE00039F500302056A903DAD12001E0F
:1004C800E49390004E123FA60FBF00010EE0FC908F
:1004D8003DAD12001EECFEE493FFEEC39F5026AE26
:1004E80009AF0A0FBF00010E903DAD12001EAE0904
:1004F800AF0AE493FC903DAD12001EE49390004EC9
:10050800123FA6ECF0AE09AF0A903DAD12001EE412
:100518009390004E123FA6E0FC903DAF12001EECF7
:10052800FCE493FDECD39D4019903DAF12001EE40E
:1005380093FC903DAD12001EE49390004E123FA62E
:10054800ECF0AE09AF0A74022FFF50010E8E098F2E
:100558000A780A740126F6500418E436F6400302B5
:1005680004B322750A00750900AE09AF0A7415BEF6
:1005780000039F5003020638903E0412001EE493C5
:1005880090004E123FA60FBF00010EE0FC903E0403
:1005980012001EECFEE493FFEEC39F5026AE09AF97
:1005A8000A0FBF00010E903E0412001EAE09AF0AEA
:1005B800E493FC903E0412001EE49390004E123F18
:1005C800A6ECF0AE09AF0A903E0412001EE4939028
:1005D800004E123FA6E0FC903E0612001EECFCE422
:1005E80093FDECD39D4019903E0612001EE493FC47
:1005F800903E0412001EE49390004E123FA6ECF0C9
:10060800AE09AF0A740F6F4E7006750A15750900AA
:10061800AE09AF0A74022FFF50010E8E098F0A78B7
:100628000A740126F6500418E436F64003020571F0
:1006380022750A00750900AE09AF0A7415BE0003D9
:100648009F5003020706903E1912001EE493900083
:100658004E123FA60FBF00010EE0FC903E1912009B
:100668001EECFEE493FFEEC39F5026AE09AF0A0FBF
:10067800BF00010E903E1912001EAE09AF0AE493A6
:10068800FC903E1912001EE49390004E123FA6EC17
:10069800F0AE09AF0A903E1912001EE49390004E86
:1006A800123FA6E0FC903E1B12001EECFCE493FDFA
:1006B800ECD39D4019903E1B12001EE493FC903E23
:1006C8001912001EE49390004E123FA6ECF0AE09FA
:1006D800AF0A740F6F4E7006750A15750900AE09DA
:1006E800AF0A74022FFF50010E8E098F0A780A7420
:1006F8000126F6500418E436F6400302063F2205A8
:100708004D22054C22054EC2CF2290F800E4936496
:1007180006600280FE75840175A70075FF8090074A
:1007280088E4F075C91075A70F75A1C775A700757E
:10073800D90075CEFF75A70F75F1FE75F2FF75F339
:100748003775F47875A4BA75A5FF75A60775AE0058
:1007580075AFFF75D48175D5FF75D6FF75D7FFC204
:1007680096C295C2A0C297E5B554BFF5B5E5B55494
:10077800DFF5B5E5B554EFF5B5E5B5547FF5B5E565
:10078800B554F7F5B5E5B554FDF5B575A70075A2EF
:100798000175A14775F80975BC0175BE0475BD6C76
:1007A80075BE0775BDA075BE0875BD0175BC007521
:1007B800BB1875BC2075BA0875E88075D11375A784
:1007C8000F75E10575E20075C7407597007597804C
:1007D800740A123F607597C0E5975420700280F83C
:1007E800758F0275A700D2AF75980075A90C75A70B
:1007F8000F75AB4375ADFB75AC1E75A700758911F8
:10080800758E00758C00758A00D2A9D28C758D0002
:10081800758B00D2ABD28E75CD0075CC0075CA0031
:1008280075CB00D2ADC2CFD2CA759104759200754E
:1008380093CD75EF0675D94075CF01900786E4F022
:10084800A3F0751300751400C299D20AC20D1204E0
:100858006474C8F51875170012257275A70FE5FBA3
:1008680090001AF0E5FA90001BF0E5F990001CF0F2
:1008780075A70090F800E493F5081226A9122BE357
:10088800900789E0900026F090078AE0900027F012
:1008980090078BE0900028F090078CE0900029F0FA
:1008A80090078DE0F56690078EE0F56890078FE079
:1008B800F569900790E0F56A900791E0F565900773
:1008C80092E0F567900793E0F564900794E0F5638C
:1008D800900795E090002AF0900796E090002BF0A2
:1008E800900797E090002CF0900798E0900041F076
:1008F800900799E0900042F090079AE0900043F04A
:1009080090079BE0900044F090079CE0900045F031
:1009180090079DE0900046F090079EE0900047F019
:1009280090079FE0900048F09007A0E0900033F017
:100938009007A1E0900034F09007A2E0900035F015
:100948009007A3E0900036F07400900082F09001C8
:100958003AE0700C90013BE0700690013CE06002C8
:100968008004C20A8002D20A90F807E4939000211A
:10097800F0900021E0440A900021F0900021E0541A
:10098800FE900021F07406900012F074029000139B
:10099800F090F802E493900014F07403900015F0BE
:1009A8007403900016F07401900017F0740590001D
:1009B80018F0900014E0B404067404900018F09045
:1009C8000014E0B403067403900018F07405900056
:1009D80019F090F804E49390001DF0740090001E44
:1009E800F090F805E49390001FF090F806E49390D7
:1009F8000020F074FF900022F07447900125F074F5
:100A08004D900126F07420900127F074349001284D
:100A1800F0744C900129F0743890012AF0743090E9
:100A2800012BF0744590012CF0742090012DF07486
:100A38002090012EF0742090012FF0743490013032
:100A4800F07453900131F07450900132F074449076
:100A58000133F090007AE0D39401400674009000CE
:100A68007AF0755801755901740390004CF0120022
:100A7800AC1204AD900014E0B404051206398003EA
:100A880012056B12259EE5B554FEF5B5900025E4D8
:100A9800F0900786E4F0A3F07524007523007548EC
:100AA80000752A00752900754900753200753100F6
:100AB800754A00755400755500755A0075510475CE
:100AC800520175343C753300757000756F0075718F
:100AD800CD7556007557007543007544007545007F
:100AE800754600755B0075470075420075410090BA
:100AF8000006E4F0A3F0900008E4F0A3F0755E00AF
:100B0800755F0090000E74FDF0A374E8F090002368
:100B1800E4F07464900024F0C200D201C202D2034F
:100B2800754D00756D00C294C293C287C290C29180
:100B3800C20C7E017F00900028E0123F8E900027B3
:100B4800E02FFF50010E90000AEEF0A3EFF09000A6
:100B580026E0700674FF900026F090000AE0FEA3DD
:100B6800E0FFEFD394FFEE940F400790000AE4F003
:100B7800A3F07400900071F07400900079F0740094
:100B8800900082F0740090008DF074009000B4F032
:100B9800E5677003756704743A90074EF074FD902A
:100BA800074FF09003D4E0900414F0D2B0D2B7D23B
:100BB800A7D2A6D2B1D2A3C207A2B6B39204A2B357
:100BC800B39205D29CD2EC75CF01A298B34005C26E
:100BD80098122F47E5136006A299B3B34002800527
:100BE800C2991234B7E51464016005E514B404022F
:100BF80080D5E54DD39405400CE55AC394C85002FE
:100C0800055A754D00E571C394FA501A786F1200B1
:100C18003FAE6FAF70EFD394E8EE940340080571D0
:100C2800757000756F00C28E7E047F00E54C123F20
:100C38008EE58D75F004A4FDACF0EF2DFDEE3CFCC7
:100C4800E58B75F04084FF7E00ED2FFFEC3EFE8EB5
:100C5800258F26D28EA2B6300401B35003020DA20E
:100C6800A2B6300401B35003020DA2A2B640670534
:100C780054A20D400575FFA0D20DE5B54401F5B5A8
:100C8800900024E4F0E554D3956640487C887D4D77
:100C9800AE25AF26123E2E8E238F24E5482FFF5017
:100CA800010E7401123F808E238F248524487554C9
:100CB80001C28E758D00758B00754C00D28E740341
:100CC800BE00039F50069000257401F0E543B4066A
:100CD80003754300D204A2B6B35003020DA2C204A6
:100CE80090006BE060181235F8A200B34008E5B533
:100CF8004408F5B58006E5B554F7F5B58002C2009D
:100D080090006EE0601812374DA202B34008E5B5B6
:100D18004402F5B58006E5B554FDF5B58006E5B5A0
:100D280054FDF5B5A207B34004D2878002C287906C
:100D38000059E06004D2908002C29090004AE0B46A
:100D48000104D2948002C294900049E0B40104D214
:100D5800938002C293A209B34004D2918002C29147
:100D6800900018E0FE900014E0C39E400990001423
:100D7800E0D39408400974FB900023F012046490B7
:100D8800001DE0601590001DE0FE900017E06E6009
:100D98000974FE900023F0120464C2CA7E017F0029
:100DA800E54E123F8EE5CD2FFF50010E8E278F287E
:100DB800D2CAE565B4014890000EE0FCA3E0FDEF5F
:100DC800C39DEE9C4039B208E52A45296013A20864
:100DD800B34008E5B54404F5B58006E5B554FBF520
:100DE800B590000EE0FEA3E0FF900010E0FCA3E049
:100DF800FDEF2DFDEE3CFC90000EECF0A3EDF0A213
:100E0800B3300501B35003020EF0A2B3300501B3AD
:100E18005003020EF0A2B35003020EE90555A20DCD
:100E2800400575FFA0D20DE5B54401F5B590002445
:100E3800E4F0E555D395685003020EE77CEA7D603F
:100E4800AE27AF28123E2E8E298F2AE569123F8ED3
:100E580074FF8E048F05FF123F708C298D2AE54997
:100E68002DFD50010C74018C068D07123F808E29D0
:100E78008F2A852A49A209B340157464123F8E90BF
:100E88000067E08E048F05FF123F708C298D2A754C
:100E9800550190000EE0FEA3E0FFAC27AD2812003C
:100EA8000390000EEEF0A3EFF0E567FF123F7074B9
:100EB8000AFF123F7090007BE08C068D07123F8E70
:100EC80074148E048F05FF123F70900010ECF0A38D
:100ED800EDF0C2CA75CD0075CC00754E00D2CAD2ED
:100EE80005A2B3B34002C205900025E0B40107E5AE
:100EF80056C394064003021501E56D902551F82864
:100F08002873900059E0C39402400302105EE55133
:100F1800D39401500302105EE55175F040A4FFAE72
:100F2800F090031212001EE0C395455018E5517564
:100F3800F040A4FFAEF090031112001EE0F52E75EC
:100F48002D0002105EE55175F040A4FFAEF090034D
:100F58001012001EE0C395454003020FFAE55175D3
:100F6800F040A4FFAEF090031112001EE55175F099
:100F780040A4FFAEF0E0FC90030F12001EECFEE070
:100F8800FFEEC39FFEE5518E0475F040A4FFAEF05E
:100F980090031012001EE0F40425458C0088F0A48C
:100FA800FFAEF0E5518F048E0575F040A4FFAEF05A
:100FB80090031212001EE55175F040A4FFAEF0E058
:100FC800FA90031012001EEAFEE0FFEEC39FFECD6A
:100FD800CCCD8E07123F70E55175F040A4FFAEF0FE
:100FE80090030F12001EE02DFD50010C8C2D8D2E4C
:100FF8008064E55175F040A4FFAEF090030F120035
:101008001EE55175F040A4FFAEF0E0FC90030E120F
:10101800001EECFEE0FFEEC39F8545F0A4FFAEF096
:10102800E5518F048E0575F040A4FFAEF0900310D3
:1010380012001EE0FECDCCCD8E07123F70E5517533
:10104800F040A4FFAEF090030E12001EE02DFD50FC
:10105800010C8C2D8D2E756D01021501900059E043
:10106800C39402400302121190004FE0D3955150EF
:10107800030211BAE55175F040A4FFAEF0900318D1
:1010880012001EE0C395455018E55175F040A4FFC5
:10109800AEF090031712001EE0F52C752B0002111C
:1010A800BAE55175F040A4FFAEF090031612001E89
:1010B800E0C395454003021156E55175F040A4FF81
:1010C800AEF090031712001EE55175F040A4FFAE74
:1010D800F0E0FC90031512001EECFEE0FFEEC39F4B
:1010E800FEE5518E0475F040A4FFAEF09003161291
:1010F800001EE0F40425458C0088F0A4FFAEF0E55E
:10110800518F048E0575F040A4FFAEF090031812BD
:10111800001EE55175F040A4FFAEF0E0FA9003160A
:1011280012001EEAFEE0FFEEC39FFECDCCCD8E0777
:10113800123F70E55175F040A4FFAEF09003151210
:10114800001EE02DFD50010C8C2B8D2C8064E55188
:1011580075F040A4FFAEF090031512001EE551751E
:10116800F040A4FFAEF0E0FC90031412001EECFE69
:10117800E0FFEEC39F8545F0A4FFAEF0E5518F0474
:101188008E0575F040A4FFAEF090031612001EE025
:10119800FECDCCCD8E07123F70E55175F040A4FF0F
:1011A800AEF090031412001EE02DFD50010C8C2BA4
:1011B8008D2CE551B40122E560D39401401BE55123
:1011C800C395565014E545C39405500D90035FE050
:1011D800A829B80006952A40028003755102E551F6
:1011E800B5602290004FE0D395514019E55175F054
:1011F80040A4FFAEF090031712001EE0A823B80029
:10120800069524400280020560756D020215019062
:101218000059E0B4022AE55175F040A4FFAEF09001
:10122800031712001EE0F52C752B00E55175F040F0
:10123800A4FFAEF090030E12001EE0F52E752D00EF
:10124800900059E0B4030F900051E0F52C752B0085
:10125800752E00752D00756D03021501E55175F0A9
:1012680040A4FFAEF090032012001EE0C3955A4040
:1012780003021338900049E07036E551D3940140D9
:1012880029AE23AF24AC2DAD2EEDD39FEC9E401A92
:10129800E55175F040A4FFAEF090031E12001EE069
:1012A800A829B80005D3952A500280021551803428
:1012B800E551D394024029AE23AF24AC2DAD2EEDD9
:1012C800D39FEC9E401AE55175F040A4FFAEF09014
:1012D800031E12001EE0A829B80005D3952A500263
:1012E80080021551E551B55236E551C39560502F2E
:1012F800E551C395565028AE23AF24AC2BAD2CEF47
:10130800D39DEE9C4019E55175F040A4FFAEF090D6
:10131800031F12001EE0A829B80006952A40028083
:10132800020551C292E55165526005C207755A001F
:10133800756D04021501E55175F040A4FFAEF090FB
:10134800031A12001EE0B40117E55175F040A4FF1E
:10135800AEF090032012001EE0240AC3955A400301
:1013680002140E753064752F00A207B3500B90005D
:1013780060E02405C39545400302140EE55175F05D
:1013880040A4FFAEF090031D12001EE0C395454037
:1013980064E55175F040A4FFAEF090031C12001EE6
:1013A800E55175F040A4FFAEF0E0FC90031B12007D
:1013B8001EECFEE0FFEEC39F8545F0A4FFAEF0E50E
:1013C800518F048E0575F040A4FFAEF090031D12F6
:1013D800001EE0FECDCCCD8E07123F70E55175F0B2
:1013E80040A4FFAEF090031B12001EE02DFD50013B
:1013F8000C8C2F8D30AE23AF24AC2FAD30EFD39DA6
:10140800EE9C4002D207756D05021501E551B40145
:1014180009900059E0C3940240030214E190035874
:10142800E0D3954550030214E1900356E0C3954577
:101438005040900357E0FE900355E0F4042EFE90D0
:101448000356E0F40425458E0088F0A4FFAEF09022
:101458000358E0FC900356E0F4042C8E048F05FF3B
:10146800123F70900355E02DFD50010C8C2B8D2CF4
:10147800802C900355E0FE900354E0F4042E85453B
:10148800F0A4FFAEF0900356E08E048F05FF123FE4
:1014980070900354E02DFD50010C8C2B8D2CE551E0
:1014A800C39560502FE551C395565028AE23AF24FD
:1014B800AC2BAD2CEFD39DEE9C4019E55175F04057
:1014C800A4FFAEF090031F12001EE0A829B8000682
:1014D800952A40028003755102900049E0B4010644
:1014E800E551640160028003755102E5516552605F
:0914F80005C207755A00756D006C
:10255100020F0A02106402121702126402133E02F1
:02256100141450
:10150100900050E02402A823B80007D3952440029C
:10151100C207900025E0B40109900059E0C394038B
:101521004003021687900049E060030215D7E55198
:10153100D394014034E55175F040A4FFAEF090031F
:101541001412001EE0A823B8001FD39524401AE509
:101551005175F040A4FFAEF090031F12001EE0A8E9
:1015610029B80005D3952A500280021551E551D3BF
:101571009401402FE55175F040A4FFAEF0900312A5
:1015810012001EE0C39545501AE55175F040A4FFC5
:10159100AEF090031E12001EE0A829B80005D395F5
:1015A1002A500280021551E551D394014021E551A1
:1015B100D39556401AE55175F040A4FFAEF0900363
:1015C1001E12001EE0A829B80005D3952A500280FA
:1015D10002155102167CE551D394024034E5517550
:1015E100F040A4FFAEF090031412001EE0A823B84F
:1015F100001FD39524401AE55175F040A4FFAEF0C9
:1016010090031F12001EE0A829B80005D3952A50A7
:101611000280021551E551D39402402FE55175F036
:1016210040A4FFAEF090031212001EE0C395455096
:101631001AE55175F040A4FFAEF090031E12001E92
:10164100E0A829B80005D3952A500280021551E57A
:1016510051D394024021E551D39556401AE5517575
:10166100F040A4FFAEF090031E12001EE0A829B8BE
:101671000005D3952A500280021551E5516552604B
:1016810005C207755A00900060E0D3954550099056
:101691000054E0C395455002C207900059E0700321
:1016A1000218EAA2A5B34008A2A4B340030218D3CA
:1016B100AE35AF367441D39F749C9E400578351288
:1016C100003FAE35AF36EFB48806EEB413028003A7
:1016D1000218B0A2A55003021773900059E0B4019B
:1016E1000B90004FE0D3956040020560900059E0F7
:1016F100B40253E55175F040A4FFAEF090032012FF
:10170100001EE0C3955A503E90004FE0D3955140E2
:1017110020E551C395565019E55175F040A4FFAE2F
:10172100F090031412001EE0A823B800069524408F
:10173100028002055190004FE0F560E5516552606D
:1017410005C207755A00900059E0B4032590004F77
:10175100E0D395514007E551C395564002800205FB
:101761005190004FE0F560E55165526005C2077583
:101771005A00A2A450030218B0900059E0B4016EBF
:10178100900049E07035E551D394014029E5517548
:10179100F040A4FFAEF090031E12001EE0A829B88D
:1017A100000FD3952A400A1551755A008551608062
:1017B1000385516080037560018033E551D3940244
:1017C1004029E55175F040A4FFAEF090031E1200D0
:1017D1001EE0A829B8000FD3952A400A1551755A61
:1017E100008551608003855160800375600290001F
:1017F10059E0D3940150030218A4E55175F040A4B7
:10180100FFAEF090032012001EE0C3955A40030280
:1018110018A4900049E07041E551D394014034E5AA
:101821005175F040A4FFAEF090031112001EE0A824
:1018310023B8001FD39524401AE55175F040A4FF49
:10184100AEF090031E12001EE0A829B80005D39542
:101851002A500280021551803FE551D39402403451
:10186100E55175F040A4FFAEF090031112001EE0A7
:10187100A823B8001FD39524401AE55175F040A460
:10188100FFAEF090031E12001EE0A829B80005D398
:10189100952A500280021551E55165526005C20733
:1018A100755A00E556B40704055E8003755E00E5D0
:1018B10063B4010EAE35AF36EF64407005EE649C43
:1018C1006002800EA2A54003755801A2A4400375D1
:1018D1005802A2A5B3B35006A2A4B3B34002800636
:1018E1007536007535000219D8A2A5B34008A2A427
:1018F100B340030219C4AE35AF367441D39F749C13
:101901009E4005783512003FAE35AF36EFB48806FC
:10191100EEB4130280030219C4A2A5406F900068BF
:10192100E0605A90004AE0B4010790004AE4F08078
:101931000690004A7401F090004AE070057560035A
:10194100800375600490004AE0B40104D2948002DF
:10195100C294E551B4041AE55175F040A4FFAEF00C
:1019610090031E12001EE0A829B80005D3952A5045
:10197100028008755103C207755A0080037560041F
:10198100E556B40704055E8003755E00A2A44033EA
:10199100900069E06021900049E0B401079000499E
:1019A100E4F080069000497401F0900049E0B40130
:1019B10004D2938002C293E556B40704055E800306
:1019C100755E00A2A5B3B35006A2A4B3B3400280D2
:1019D10006753600753500E5586559600690008238
:1019E100E06003021B60C29C751400751300C2CA3B
:1019F100E558902563F82828738012122BE3800D97
:0D1A0100122CBC8008122D958003122E6E51
:0F2563000219FA0219FC021A01021A06021A0BD7
:101A0E00900029E090007AF0E566900057F0E568C6
:101A1E00900062F0E569900063F0E56A900074F062
:101A2E00E56590007CF0E56790007DF0E564900040
:101A3E0080F0E563900081F090002AE090013AF08A
:101A4E0090002BE090013BF090002CE090013CF0D8
:101A5E00900041E0900090F0900042E0900091F0F4
:101A6E00900043E0900092F0900044E0900093F0DC
:101A7E00900045E0900094F0900046E0900095F0C4
:101A8E00900047E0900096F0900048E0900097F0AC
:101A9E00900033E0900099F0900034E090009AF0BE
:101AAE00900035E090009BF0900036E090009CF0A6
:101ABE007400900082F07447900125F0744D9001EF
:101ACE0026F07420900127F07434900128F0744CA5
:101ADE00900129F0743890012AF0743090012BF0A7
:101AEE00744590012CF0742090012DF0742090011B
:101AFE002EF0742090012FF07434900130F0745356
:101B0E00900131F07450900132F07444900133F032
:101B1E009003D4E0900414F0743A90074EF074FDE4
:101B2E0090074FF01200AC900004E4F0A3F0900088
:101B3E00067475F0A37430F09000087475F0A374F9
:101B4E0030F0855859D2CA754C00D29C741B900047
:101B5E0023F0E556C394065005E551B55202804E6A
:101B6E00C207E55175F040A4FFAEF09003221200BB
:101B7E001EE030E003D38001C39296E55175F0402C
:101B8E00A4FFAEF090032312001EE030E003D380DA
:101B9E0001C39295855152AE29AF2A7405BE00033A
:101BAE009F5007E545D3940550028002D292E55628
:101BBE00D394055003021C85C207E551D39401400E
:101BCE0059E55175F040A4FFAEF090031E12001EB1
:101BDE00E0A829B80007D3952A40021551E55165B2
:101BEE00526035E55175F040A4FFAEF0900322121D
:101BFE00001EE030E003D38001C39296E55175F0EC
:101C0E0040A4FFAEF090032312001EE030E003D399
:101C1E008001C39295855152805DE556B4061A90A7
:101C2E0000ACE030E003D38001C392969000ADE0AB
:101C3E0030E003D38001C39295E556B4071A9000A5
:101C4E00A5E030E003D38001C392969000A6E03069
:101C5E00E003D38001C39295E556B4081A90009E16
:101C6E00E030E003D38001C3929690009FE030E015
:101C7E0003D38001C39295900072E06058E54575DC
:101C8E00F00284FF7E0090014E12001EE0F55CE52E
:101C9E004775F00A84FF7E0090024E12001EE0F59A
:101CAE005DE55C255DD39464400BE55C255DC394D6
:101CBE0064F55C8003755C00E55C75F00284FF7E64
:101CCE00008F5CEFC394335007EF24CDF55C800397
:101CDE00755CFF801CE54575F00284FF7E00900167
:101CEE004E12001EE075F00284FF7E00EF24CDF54B
:101CFE005CE595C3955C4004C2A28002D2A2A20705
:101D0E00B34005E556B407037571CDE595C39571DE
:101D1E004004C2A18002D2A1E543C394064003024F
:101D2E002329A2EDB35003022329C2EDE54360033C
:101D3E00021E8B7E017F00E5BE123F8EE5BD2FFF9A
:101D4E0050010E900000EEF0A3EFF0900029E0B4E9
:101D5E0001177E0F7FFF900000E0FCA3E0FD120054
:101D6E0003900000EEF0A3EFF0900079E0B4025B78
:101D7E00900000E0FEA3E0FF90000AE0FCA3E0FD6F
:101D8E00EDD39FEC9E400F900000E0F8A3E0900092
:101D9E000AC8F0A3C8F0900000E0FEA3E0FF900098
:101DAE000CE0FCA3E0FDEFD39DEE9C400F900000F5
:101DBE00E0F8A3E090000CC8F0A3C8F0900000E09B
:101DCE00FEA3E0FF7404123F808F44900079E07010
:101DDE0060900000E0FEA3E0FF90000AE0FCA3E0AC
:101DEE00FDEFD39DEE9C400D120003900000EEF02F
:101DFE00A3EFF08007900000E4F0A3F0900000E065
:101E0E00FEA3E0FF7410123F8E900026E08E048F2A
:101E1E0005FF123F70900000ECF0A3EDF07400D3BC
:101E2E009D74019C4008900001E0F54480037544C8
:101E3E00FFE54475F00AA4FFAEF074198E048F0509
:101E4E00FF123F708D45ED2532FFAE3150010E74FD
:101E5E0001123F808F45854532753100EFD3946274
:101E6E004003754562900072E06401600690006662
:101E7E00E060028005754301800375BB17E543B42E
:101E8E0001028003021F7B7E017F00E5BE123F8EA2
:101E9E00E5BD2FFF50010E900000EEF0A3EFF09085
:101EAE000072E0B4017EE53445336025AC33AD34C9
:101EBE001DBDFF011C8F028E038C068D07903C43C7
:101ECE0012002EE493FE740193FFEFC39AEE9B4033
:101EDE000280057833123FB8AE33AF3474B3BE0010
:101EEE0025D39F4021900000E0FCA3E0FD0FBF0032
:101EFE00010E903C4312002EE493FE740193FFED0D
:101F0E00C39FEC9E40028005783312003FAE33AF84
:101F1E0034E56A123F8E74648E048F05FF123F7093
:101F2E008D478033900066E0602D900000E0FEA3A8
:101F3E00E0FFEFD39400EE9408400F900066E0B4FB
:101F4E000104C2098002D209800D900066E0B4013E
:101F5E0004D2098002C209900072E0640260069009
:101F6E000066E0600575BB168003754302E543B459
:101F7E00020280030220697E017F00E5BE123F8EC1
:101F8E00E5BD2FFF50010E900000EEF0A3EFF09094
:101F9E000072E0B4027EE53445336025AC33AD34D7
:101FAE001DBDFF011C8F028E038C068D07903AD942
:101FBE0012002EE493FE740193FFEFC39AEE9B4042
:101FCE000280057833123FB8AE33AF3474B3BE001F
:101FDE0025D39F4021900000E0FCA3E0FD0FBF0041
:101FEE00010E903AD912002EE493FE740193FFED88
:101FFE00C39FEC9E40028005783312003FAE33AF94
:10200E0034E56A123F8E74648E048F05FF123F70A2
:10201E008D478033900066E0602D900000E0FEA3B7
:10202E00E0FFEFD39400EE9408400F900066E0B40A
:10203E000104C2098002D209800D900066E0B4014D
:10204E0004D2098002C209900072E0700375470045
:10205E00900066E07002C20975BB1FE543B40345EC
:10206E007E017F00E5BE123F8EE5BD2FFF50010EB3
:10207E00900000EEF0A3EFF07409123F8E74E68E1E
:10208E00048F05FF123F708C418D42E54A2DFD50A5
:10209E00010C74018C068D07123F808E418F428594
:1020AE00424A75BB19E543B4040280030222117E35
:1020BE00017F00E5BE123F8EE5BD2FFF50010E9051
:1020CE000000EEF0A3EFF07404123F808F4BE56436
:1020DE00B40102800302219E756B00756B00E56BE7
:1020EE00D39407400302218BE56B900041123FA66B
:1020FE00E0D3954B501AE56B900041123FA6E0F4E9
:10210E0004254BFEE56B900037123FA6EEF08017CC
:10211E00E56B900041123FA6E0C3954BFEE56B9038
:10212E000037123FA6EEF0E56BC394044009900011
:10213E0084E0C3956B503BE56B6029E56B900037EF
:10214E00123FA6FEE0FFEE90003FE0D39F4013E566
:10215E006B900037123FA6E090003FF0E56B9000C9
:10216E0040F0800E900037E090003FF07400900039
:10217E0040F0786B740126F640030220EC9000408C
:10218E00E0F4042408F556E556D394054002C292B5
:10219E00E564D39401402FE54BD3946E4004D20EE8
:1021AE008002C20E755605E564B40205A20EB34058
:1021BE00028003755607E564B40306A20EB3B3405E
:1021CE00028003755607E55765566008E55104F51C
:1021DE0052855657E556B40708E5B54480F5B580E7
:1021EE0006E5B5547FF5B5E55664066005E556B4CB
:1021FE000808E5B54410F5B58006E5B554EFF5B51C
:10220E0075BB13E543B4050280030223257E017FCF
:10221E0000E5BE123F8EE5BD2FFF50010E9000006F
:10222E00EEF0A3EFF07404123F808F46E563B40224
:10223E00028003022322756B00756B00E56BD3944D
:10224E000340030222D9E56B900033123FA6E0D380
:10225E009546501AE56B900033123FA6E0F4042524
:10226E0046FEE56B90002D123FA6EEF08017E56B53
:10227E00900033123FA6E0C39546FEE56B90002D0D
:10228E00123FA6EEF0E56B6029E56B90002D123F34
:10229E00A6FEE0FFEE900031E0D39F4013E56B9079
:1022AE00002D123FA6E0900031F0E56B900032F069
:1022BE00800E90002DE0900031F07400900032F00E
:1022CE00786B740126F6400302224A900082E07079
:1022DE0043E52A45296036E558C39403500A900019
:1022EE0032E004C3940340028007900032E004F50C
:1022FE0058E558D39402400A900032E004D3940279
:10230E0050028007900032E004F5588007900032AA
:10231E00E004F55875BB180543D2ECE55ED3940482
:10232E00500302241175CF01C2A2AE35AF367488A8
:10233E00D39F74139E4005A2A5B34014AE35AF369D
:10234E007488D39F74139E4005A2A4B340028048A4
:10235E00783512003FAE35AF36EFB4883BEEB4138E
:10236E0037A2A5B3500990004FE0D395515002808B
:10237E000405518011A2A5B3500890004FE065519D
:10238E0060028002D207A2A4B35007E551D3940194
:10239E00500280041551C207A2A5B3B35006A2A4E1
:1023AE00B3B340028006753600753500E5516552AF
:1023BE006035E55175F040A4FFAEF0900322120097
:1023CE001EE030E003D38001C39296E55175F040D4
:1023DE00A4FFAEF090032312001EE030E003D38082
:1023EE0001C39295855152A20740057571CD8003A8
:1023FE007571FFE595C395714004C2A18002D2A10B
:10240E00022333A20DB3500DAE25AF2674E8C39F41
:10241E0074039E4002800575FFA0D20DAE25AF2637
:10242E00EFD39420EE944E5003022525120464C27D
:10243E008E758D00758B00754C00D28EC20775702F
:10244E0000756F007571CD755104752400752300EC
:10245E00755400755A00C287900059E06004D290FE
:10246E008002C29090004AE0B40104D2948002C26D
:10247E0094900049E0B40104D2938002C293A20961
:10248E00B34004D2918002C29190006BE0601812AA
:10249E0035F8A200B34008E5B54408F5B58006E569
:1024AE00B554F7F5B58002C20090006EE0601812C8
:1024BE00374DA202B34008E5B54402F5B58006E5F6
:1024CE00B554FDF5B58006E5B554FDF5B590000E95
:1024DE0074FDF0A374E8F0E543B406037543009071
:1024EE000025E4F0752600752500758D00758B00AE
:1024FE00754C00900024E0C394035008900024E033
:10250E0004F080067403900024F0900024E0B403DD
:10251E0006E5B554FEF5B5AE27AF28EFD39410EE11
:10252E009427401CC2CA75CD0075CC007528007565
:10253E002700D2CA754E00752A0075290075550000
:03254E00020BCFAE
:1038FF0000000100013201640196019602000212DC
:10390F0002240200020003000340038003C00400EE
:10391F000440048004C005000600060006000600EF
:10392F00060006000600060000FF01310163019545
:10393F0001FF01FF0211022302FF02FF02FF033FFB
:10394F00037F03BF03FF043F047F04BF04FF05FF92
:10395F0006FF06FF06FF06FF06FF06FF06FF06FF30
:10396F000FAA0FA50F9F0F9A0F940F8D0F870F8020
:10397F000F780F710F680F600F570F4E0F450F3BEA
:10398F000F300F250F1A0F0E0F020EF50EE80EDB7C
:10399F000ECC0EBE0EAE0E9F0E8E0E7D0E6C0E5A00
:1039AF000E470E340E200E0C0DF70DE20DCB0DB59C
:1039BF000D9D0D850D6D0D540D3A0D200D050CE966
:1039CF000CCE0CB10C940C760C580C3A0C1B0BFB58
:1039DF000BDB0BBB0B9A0B790B570B350B130AF148
:1039EF000ACE0AAB0A870A640A400A1C09F809D4EE
:1039FF0009B0098C09670943091F08FB08D608B2EB
:103A0F00088E086A0846082307FF07DC07B90796E0
:103A1F0007730751072F070D06EC06CA06AA06897A
:103A2F0006690649062A060A05EC05CD05B005927A
:103A3F0005750558053C0520050504EA04CF04B5B6
:103A4F00049C04820469045104390422040B03F416
:103A5F0003DE03C803B2039D038903750361034D9E
:103A6F00033B03280316030402F202E102D102C052
:103A7F0002B002A00291028202730265025702494C
:103A8F00023C022F02220216020901FD01F201E699
:103A9F0001DB01D001C601BB01B101A7019D01945A
:103AAF00018B018201790170016801600158015099
:103ABF000148014101390132012B0125011E011875
:103ACF000111010B010500FF00FA0FA60FA00F99BE
:103ADF000F920F8B0F840F7C0F740F6B0F620F58A9
:103AEF000F4E0F430F380F2C0F1F0F120F050EF72E
:103AFF000EE80ED80EC80EB70EA50E930E800E6CE4
:103B0F000E580E420E2C0E150DFD0DE40DCB0DB102
:103B1F000D950D790D5D0D3F0D200D010CE10CC0C4
:103B2F000C9E0C7C0C590C350C100BEA0BC40B9E25
:103B3F000B760B4F0B260AFD0AD40AAA0A800A55E8
:103B4F000A2A09FF09D409A8097C0950092508F98F
:103B5F0008CD08A10875084A081E07F307C8079D76
:103B6F0007730749072006F706CE06A6067E0657F7
:103B7F000630060A05E405BF059B05770554053297
:103B8F00051004EF04CE04AE048F04710453043502
:103B9F00041903FD03E203C703AD0394037B03631F
:103BAF00034B0334031E030802F302DE02CA02B6FC
:103BBF0002A30291027F026D025C024C023C022CB6
:103BCF00021D020E020001F201E401D701CA01BE7B
:103BDF0001B101A6019A018F0185017A0170016679
:103BEF00015D0153014A01410139013101290121CF
:103BFF0001190112010B010400FD00F700F000EAAA
:103C0F0000E400DE00D900D300CE00C900C400BF1D
:103C1F0000BA00B500B100AD00A800A400A0009C40
:103C2F00009900950091008E008A00870084008122
:043C3F00007E007B88
:10257200751A00751900AE19AF1AAC17AD18EDC374
:102582009FEC9E401674FF123F6075CF01781A745B
:102592000126F6500418E436F650DB22900786E452
:1025A200F0A3F0751000750F00751300751400C2CA
:1025B2000FD21022C2AF75D900758F0375B7A575FA
:1025C200B7F190F800E4F0758F0175B7A575B7F112
:1025D200E50890F800F075B7A575B7F190F801E439
:1025E200F075B7A575B7F190079DE090F802F07508
:1025F200B7A575B7F19007A1E090F803F075B7A5FC
:1026020075B7F190079EE090F804F075B7A575B71D
:10261200F190079FE090F805F075B7A575B7F190B6
:1026220007A0E090F806F075B7A575B7F19007A27C
:10263200E090F807F0758F0075D940D2AF2290076D
:1026420088E0B4AB61C2AF75D90075B62275F522C8
:10265200758F0375B7A575B7F1740090F600F07524
:102662008F01750A00750900AE09AF0A7413BE0026
:10267200279F402475B7A575B7F190078912001EF0
:10268200E0FC90F60012001EECF0780A740126F6C7
:10269200500418E436F650D0758F0075F51175B6F2
:1026A2002075D940D2AF22C2AF75D90075F5227517
:1026B2000A00750900AE09AF0A7413BE00229F40DA
:1026C2001F90F60012001EE493FC90078912001E70
:1026D200ECF0780A740126F6500418E436F650D568
:1026E20075F51175D940D2AF22900788E0B4AA02DD
:1026F2008003022828C2AF75D90075B62275F5226B
:10270200758F0375B7A575B7F1740090EE00F0757B
:10271200B7A575B7F1740090F000F075B7A575B75D
:10272200F1740090F200F075B7A575B7F1740090DE
:10273200F400F0758F01750A00750900AE09AF0A41
:1027420074FFC39F74019E402475B7A575B7F190BD
:10275200004E12001EE0FC90EE0012001EECF0781B
:102762000A740126F6500418E436F650CF750A00B2
:10277200750900AE09AF0A74FFC39F74019E40241D
:1027820075B7A575B7F190024E12001EE0FC90F0ED
:102792000012001EECF0780A740126F6500418E4C8
:1027A20036F650CF750A00750900AE09AF0A74FFFC
:1027B200C39F74019E402475B7A575B7F190044E6E
:1027C20012001EE0FC90F20012001EECF0780A7477
:1027D2000126F6500418E436F650CF750A00750942
:1027E20000AE09AF0A74FFC39F74019E402475B7FF
:1027F200A575B7F190064E12001EE0FC90F400128F
:10280200001EECF0780A740126F6500418E436F63D
:1028120050CF758F0075F51175B62075D940D2AFBE
:10282200743A90074EF022900788E0B4AA0280031F
:10283200022966C2AF75D90075B62275F522758F69
:102842000375B7A575B7F1740090E600F075B7A5EA
:1028520075B7F1740090E800F075B7A575B7F1741B
:102862000090EA00F075B7A575B7F1740090EC001E
:10287200F0758F01750A00750900AE09AF0A74FF81
:10288200C39F74019E402475B7A575B7F190004EA1
:1028920012001EE0FC90E60012001EECF0780A74B2
:1028A2000126F6500418E436F650CF750A00750971
:1028B20000AE09AF0A74FFC39F74019E402475B72E
:1028C200A575B7F190024E12001EE0FC90E80012CE
:1028D200001EECF0780A740126F6500418E436F66D
:1028E20050CF750A00750900AE09AF0A74FFC39F85
:1028F20074019E402475B7A575B7F190044E12007D
:102902001EE0FC90EA0012001EECF0780A74012628
:10291200F6500418E436F650CF750A00750900AE79
:1029220009AF0A74FFC39F74019E402475B7A57551
:10293200B7F190064E12001EE0FC90EC0012001E51
:10294200ECF0780A740126F6500418E436F650CFFB
:10295200758F0075F51175B62075D940D2AF743AEE
:1029620090074EF022900788E0B4AA028003022A60
:10297200A4C2AF75D90075B62275F522758F03759D
:10298200B7A575B7F1740090DE00F075B7A575B7FD
:10299200F1740090E000F075B7A575B7F17400907E
:1029A200E200F075B7A575B7F1740090E400F07518
:1029B2008F01750A00750900AE09AF0A74FFC39F43
:1029C20074019E402475B7A575B7F190004E1200B0
:1029D2001EE0FC90DE0012001EECF0780A74012664
:1029E200F6500418E436F650CF750A00750900AEA9
:1029F20009AF0A74FFC39F74019E402475B7A57581
:102A0200B7F190024E12001EE0FC90E00012001E90
:102A1200ECF0780A740126F6500418E436F650CF2A
:102A2200750A00750900AE09AF0A74FFC39F7401ED
:102A32009E402475B7A575B7F190044E12001EE0B2
:102A4200FC90E20012001EECF0780A740126F650A7
:102A52000418E436F650CF750A00750900AE09AFC6
:102A62000A74FFC39F74019E402475B7A575B7F120
:102A720090064E12001EE0FC90E40012001EECF0E4
:102A8200780A740126F6500418E436F650CF758F92
:102A92000075F51175B62075D940D2AF743A90071A
:102AA2004EF022900788E0B4AA028003022BE2C211
:102AB200AF75D90075B62275F522758F0375B7A566
:102AC20075B7F1740090D600F075B7A575B7F174BB
:102AD2000090D800F075B7A575B7F1740090DA00D0
:102AE200F075B7A575B7F1740090DC00F0758F0131
:102AF200750A00750900AE09AF0A74FFC39F74011D
:102B02009E402475B7A575B7F190004E12001EE0E5
:102B1200FC90D60012001EECF0780A740126F650E2
:102B22000418E436F650CF750A00750900AE09AFF5
:102B32000A74FFC39F74019E402475B7A575B7F14F
:102B420090024E12001EE0FC90D80012001EECF023
:102B5200780A740126F6500418E436F650CF750A46
:102B620000750900AE09AF0A74FFC39F74019E404D
:102B72002475B7A575B7F190044E12001EE0FC90C3
:102B8200DA0012001EECF0780A740126F6500418DE
:102B9200E436F650CF750A00750900AE09AF0A7423
:102BA200FFC39F74019E402475B7A575B7F19006C7
:102BB2004E12001EE0FC90DC0012001EECF0780ABF
:102BC200740126F6500418E436F650CF758F00755E
:102BD200F51175B62075D940D2AF743A90074EF010
:102BE20022C2AF75D90075F522750A00750900AECB
:102BF20009AF0A74FFC39F74019E401F90EE00123A
:102C0200001EE493FC90004E12001EECF0780A7451
:102C12000126F6500418E436F650D4750A007509F8
:102C220000AE09AF0A74FFC39F74019E401F90F06B
:102C32000012001EE493FC90024E12001EECF0788B
:102C42000A740126F6500418E436F650D4750A00C8
:102C5200750900AE09AF0A74FFC39F74019E401F3D
:102C620090F20012001EE493FC90044E12001EEC3F
:102C7200F0780A740126F6500418E436F650D4753A
:102C82000A00750900AE09AF0A74FFC39F74019E62
:102C9200401F90F40012001EE493FC90064E1200B6
:102CA2001EECF0780A740126F6500418E436F65049
:102CB200D475F51175D940D2AF22C2AF75D900755E
:102CC200F522750A00750900AE09AF0A74FFC39FA9
:102CD20074019E401F90E60012001EE493FC9000D7
:102CE2004E12001EECF0780A740126F6500418E425
:102CF20036F650D4750A00750900AE09AF0A74FFA2
:102D0200C39F74019E401F90E80012001EE493FCD2
:102D120090024E12001EECF0780A740126F650045E
:102D220018E436F650D4750A00750900AE09AF0AE8
:102D320074FFC39F74019E401F90EA0012001EE4BC
:102D420093FC90044E12001EECF0780A740126F6F1
:102D5200500418E436F650D4750A00750900AE091D
:102D6200AF0A74FFC39F74019E401F90EC001200D3
:102D72001EE493FC90064E12001EECF0780A7401D9
:102D820026F6500418E436F650D475F51175D9407C
:102D9200D2AF22C2AF75D90075F522750A00750946
:102DA20000AE09AF0A74FFC39F74019E401F90DEFC
:102DB2000012001EE493FC90004E12001EECF0780C
:102DC2000A740126F6500418E436F650D4750A0047
:102DD200750900AE09AF0A74FFC39F74019E401FBC
:102DE20090E00012001EE493FC90024E12001EECD2
:102DF200F0780A740126F6500418E436F650D475B9
:102E02000A00750900AE09AF0A74FFC39F74019EE0
:102E1200401F90E20012001EE493FC90044E120048
:102E22001EECF0780A740126F6500418E436F650C7
:102E3200D4750A00750900AE09AF0A74FFC39F7406
:102E4200019E401F90E40012001EE493FC90064E87
:102E520012001EECF0780A740126F6500418E436CB
:102E6200F650D475F51175D940D2AF22C2AF75D9DB
:102E72000075F522750A00750900AE09AF0A74FFE4
:102E8200C39F74019E401F90D60012001EE493FC63
:102E920090004E12001EECF0780A740126F65004DF
:102EA20018E436F650D4750A00750900AE09AF0A67
:102EB20074FFC39F74019E401F90D80012001EE44D
:102EC20093FC90024E12001EECF0780A740126F672
:102ED200500418E436F650D4750A00750900AE099C
:102EE200AF0A74FFC39F74019E401F90DA00120064
:102EF2001EE493FC90044E12001EECF0780A74015A
:102F020026F6500418E436F650D4750A0075090006
:102F1200AE09AF0A74FFC39F74019E401F90DC008C
:102F220012001EE493FC90064E12001EECF0780A8A
:102F3200740126F6500418E436F650D475F511756E
:102F4200D940D2AF22E51464046006E59964FF60BB
:102F5200028031A20F4004D20F8027E5146008746A
:102F6200E62514900023F0E513600874F025139011
:102F72000023F0E514B4010280FE751400751300FD
:102F8200C20F8002C20FE5149038A2F82828737588
:102F92001400E599B4FF03751301E599B4FE0375B6
:102FA2001302E599B4FD03751303E599B4FC0375A7
:102FB2001304E599B4FA03751305E599B4FB067594
:102FC2001401120464E599B4F90675140412046438
:102FD200E599D394E54007E599C394F04002801641
:102FE2008599157514027E017F00E515C394E612DA
:102FF2003F8E8E0D8F0E900786E4F0A3F0E599D3F5
:1030020094C44007E599C394E64002802885991547
:1030120075140374E5C39515F50E750D00AE0DAF6D
:103022000E9038FF12002EE493F8740193900786F5
:10303200C8F0A3C8F0D2990234B6900786E0FEA386
:10304200E0FFEFC39400EE94054009EFD394FFEE46
:1030520094064013900786E0FEA3E0FF90004E1214
:10306200001EE599F0800385996C90078612000E88
:10307200900786E0FEA3E0FFEFB40106EEB407027C
:1030820080030232C690074EE0B43C028003023253
:10309200C6A20AB35005A20BB340030231B9C29CC7
:1030A20090007AE090078CF0900057E090078DF046
:1030B200900062E090078EF0900063E090078FF03E
:1030C200900074E0900790F090007CE0900791F0FF
:1030D20090007DE0900792F0900080E0900793F0DE
:1030E200900081E0900794F090013AE0900795F00B
:1030F20090013BE0900796F090013CE0900797F03A
:10310200900090E0900798F0900091E0900799F07D
:10311200900092E090079AF0900093E090079BF065
:10312200900094E090079CF0900095E090079DF04D
:10313200900096E090079EF0900097E090079FF035
:10314200900099E09007A0F090009AE09007A1F01B
:1031520090009BE09007A2F090009CE09007A3F003
:103162007400900082F01200AC74AB900788F012E9
:0A317200264074AA900788F0E55883
:0638A200022F9102303CF0
:10317C009038C3F828287380121226EB800D122881
:0B318C002980081229678003122AA581
:0F38C30002318302318502318A02318F02319442
:10319700900788E4F090013AE0700C90013BE070F2
:1031A7000690013CE060028004C20A8002D20A0253
:1031B70032BBC29C900078E0900789F090005EE0F7
:1031C70090078AF090005FE090078BF090007AE01C
:1031D70090078CF0900057E090078DF0900062E028
:1031E70090078EF0900063E090078FF0900074E0F6
:1031F700900790F090007CE0900791F090007DE0C0
:10320700900792F0900080E0900793F0900081E0A3
:10321700900794F090013AE0900795F090013BE019
:10322700900796F090013CE0900797F0900090E0AF
:10323700900798F0900091E0900799F0900092E045
:1032470090079AF0900093E090079BF0900094E02D
:1032570090079CF0900095E090079DF0900096E015
:1032670090079EF0900097E090079FF0900099E0FC
:103277009007A0F090009AE09007A1F090009BE0E3
:103287009007A2F090009CE09007A3F074009000D4
:1032970082F074AB900788F012264074AA900788D2
:1032A700F01226EB122829122967122AA5D29C753B
:1032B70099FB80FED29C7514007513007599FB026B
:1032C70034B6900786E0FEA3E0FFEF4E70068599BF
:1032D70010750F00900786E0FEA3E0FF74016F4EA4
:1032E700701BAC0FAD10AA0DAB0EED2BFBEC3AFA31
:1032F7008A068B0790004E12001EE599F09007860C
:1033070012000E900786E0FEA3E0FF74026F4E7076
:103317000C1200AC8515997514007513000234B6AC
:10332700900786E0FEA3E0FF90004E12001EE5998D
:10333700F090078612000E900786E0FEA3E0FFAC30
:103347000DAD0E8F028E038C068D07903937120054
:103357002EE493F9740193FEEAD39EEB9940098515
:1033670015997514007513000234B6900786E0FEB0
:10337700A3E0FF90004E12001EE599F09007861219
:10338700000E900786E0FEA3E0FFEFB40006EEB460
:10339700010280030234B690001CE0D394C7400BAF
:1033A70090001CE0C394C8F516801A90001CE0D367
:1033B7009463400B90001CE0C39464F5168006905C
:1033C700001CE0F516E51675F002A4FFAEF08F6B52
:1033D700EF90004E123FA6EFFCE0FDEC900051127B
:1033E7003FA6EDFCE0FDEC2DB5160280030234A8E4
:1033F7000FEF90004E123FA6E56BFFE0FCEF900049
:1034070052123FA6ECFFE0FCEFC39CB51602800307
:103417000234A8E56B900050123FA6E56BFFE0FC75
:10342700EF900053123FA6ECFFE0FCEF2CB51671AE
:10343700E56B900054123FA6E0C3951690079DF0E8
:10344700E56B900055123FA6E0C3951690079EF0D6
:10345700E56B900058123FA6E0C3951690079FF0C2
:10346700E56B900059123FA6E0C395169007A0F0B0
:10347700E56B90005A123FA6E0C395169007A1F09E
:10348700E56B90005B123FA6E0C395169007A2F08C
:103497001225B67599F9751864751700122572808B
:0F34A700FE7599FF75186475170012257280FE67
:0938A8000232C902332702337217
:1034B60022E5139038B1F82828730235F79007866D
:1034C600E0FEA3E0FF90001212001EE0F5999007BF
:1034D6008612000E900786E0FEA3E0FF74116F4E81
:1034E60070037513000235F78562990235F7900768
:1034F60086E0FEA3E0FF90004E12001EE0F599EF75
:10350600B40107EEB4070375130090078612000E88
:073516000235F7900787E082
:0F38B1000234C00234C30234EE0234F40235197B
:10351D009038D2F82828738524990235EC852A999C
:10352D000235EC8544990235EC8547990235EC85D9
:10353D0051990235EC8560990235EC855699023525
:10354D00EC8558990235EC756E00900069E07006B7
:10355D00900068E060028016A2A44006E56E440467
:10356D00F56EA2A54006E56E4402F56E801A900038
:10357D004AE0B40106E56E4410F56E900049E0B4E2
:10358D000106E56E4420F56EA207B34006E56E44D4
:10359D0001F56EA209B34006E56E4408F56E856E21
:1035AD0099803CA210B340077599FAC2108017A2FA
:1035BD000CB3400575990F800B900023E0F59990A1
:1035CD000023E4F0C20C80178542998012854B9937
:0F35DD00800D85469980087599FC800375130051
:1038D20002352402352A02353002353602353C02E1
:1038E200354202354802354E0235540235B00235B2
:0D38F200D50235DA0235DF0235E40235E992
:0B35EC0090078612000E8003120048BA
:0338C0000235F4DA
:1035F7002290006BE0B4010385241190006BE0B4C6
:103607000203852A1190006BE0B4030385441190EF
:10361700006BE0B4040385471190006BE0B4050329
:1036270085511190006BE0B4060385561190006B2D
:10363700E0B4070385581190006CE0FE90006DE040
:10364700C39E50030236CE90006BE0D39404402C07
:1036570090006CE0D39511500990006DE0C395116F
:1036670050028002D20090006CE0D395115009906F
:10367700006DE0C395115002C200804990006BE0D5
:10368700B4041890006DE0C395115002D200900069
:103697006CE0D395114002C200802A90006CE0C311
:1036A7009511500990006DE0D3951150028002D218
:1036B7000090006CE0D39511500990006DE0C39520
:1036C700115002C200807E90006BE0D39404402C1E
:1036D70090006CE0C39511400990006DE0D39511FF
:1036E70040028002C20090006CE0C395114009902F
:1036F700006DE0D395114002D200804990006BE045
:10370700B4041890006CE0C395115002C2009000F9
:103717006DE0D395114002D200802A90006CE0C37F
:103727009511400990006DE0D395114002D20090A9
:10373700006CE0D39511400990006DE0C3951140EE
:10374700028002C2002290006EE0B40103852411BA
:1037570090006EE0B40203852A1190006EE0B40376
:103767000385441190006EE0B4040385471190006F
:103777006EE0B4050385511190006EE0B406038531
:10378700561190006EE0B4070385581190006FE062
:10379700FE900070E0C39E500302382390006EE055
:1037A700D39404402C90006FE0D3951150099000FA
:1037B70070E0C3951150028002D20290006FE0D3EF
:1037C70095115009900070E0C395115002C2028014
:1037D7004990006EE0B40418900070E0C395115052
:1037E70002D20290006FE0D395114002C202802AF4
:1037F70090006FE0C395115009900070E0D39511C8
:1038070050028002D20290006FE0D39511500990C8
:103817000070E0C395115002C202807E90006EE0F6
:10382700D39404402C90006FE0C395114009900099
:1038370070E0D3951140028002C20290006FE0C38E
:1038470095114009900070E0D395114002D2028093
:103857004990006EE0B4041890006FE0C3951150D2
:1038670002C202900070E0D395114002D202802A72
:1038770090006FE0C395114009900070E0D3951157
:103887004002D20290006FE0D3951140099000707A
:0B389700E0C3951140028002C2022233
:093FA6002582F5825002058322F8
:10002E00EF2F500205832582F582E5833E2EF58360
:01003E00229F
:08000300C3EF9DFFEE9CFE22FD
:08003F000806B60002180622B3
:0D000E00A3E004F07006123F9CE004F02215
:083FB8000816B6FF02181622DC
:0E3F8000048007C3CE13CECF13CFD5E0F622B8
:103E2E00BC000FBE0008ED8FF084FFADF022E4FE63
:103E3E00FF22BE000DEF60FE54F0606F20E703021C
:103E4E003EE4EAC0E0EBC0E078017A0075F001EEE6
:103E5E0020E710EF25E0FFEE33FE0AC5F023C5F094
:103E6E0030E7F0EA5407F9096A7A007B006001082E
:103E7E00C3EC9E40167004ED9F4010ED9FFDEC9E2E
:103E8E00FCE5F0CA4ACA03F5F08005E5F003F5F04B
:103E9E00C3EE13FEEF13FFD9D77908CACBCAD8D019
:103EAE00EAFEEBFFD0E0FBD0E0FA22EC8FF084FCD0
:103EBE00ED54F045F0C48FF084FEEDC454F045F09F
:103ECE00C48FF084FDEEC4FE54F02DFFEE540F3C73
:103EDE00FEADF07C0022790078008FF0EC7E082099
:103EEE00E70DC3CD33CD33C933C9C833C8DEF08433
:103EFE0049F9E5F08FF0BE00E6FD7C00E9FFE8FE33
:013F0E002290
:0E3F8E00F88FF0A4FFE5F0CE88F0A42EFE22FE
:103F6000600D782B023F6A007830D8FED5E0F82249
:103F7000EEC0E07E00123E2EEFFDEEFCD0E0FE2211
:03000B00023F0FA2
:03001B00023F2A77
:03002B00023F454C
:03000000023FAF0D
:093FAF0075817275D00002071241
:0B001E00E5822FF582E5833EF583228A
:0A3F9C000582D582021583158222EA
:103F0F00C0E0C0F0C083C082C0D075D000120707D8
:103F1F00D0D0D082D083D0F0D0E032C0E0C0F0C09B
:103F2F0083C082C0D075D00012070AD0D0D082D003
:103F3F0083D0F0D0E032C0E0C0F0C083C082C0D0E8
:103F4F0075D00012070DD0D0D082D083D0F0D0E042
:013F5F00322F
:00000001FF
